
 Start         Length     Name                   Class
 0001:00401000 00013FE8H .text                   CODE
 0002:00415000 00000214H .itext                  ICODE
 0003:00416000 00000284H .data                   DATA
 0004:00417000 000000B4H .bss                    BSS
 0005:00000000 00000000H .tls                    TLS


Detailed map of segments

 0001:00000000 000001D6 C=CODE     S=.text    G=(none)   M=System   ACBP=A9
 0001:000001D8 00000016 C=CODE     S=.text    G=(none)   M=TypInfo  ACBP=A9
 0001:000001F0 0000006E C=CODE     S=.text    G=(none)   M=SysUtils ACBP=A9
 0001:00000260 0000025C C=CODE     S=.text    G=(none)   M=Windows  ACBP=A9
 0001:000004BC 00000036 C=CODE     S=.text    G=(none)   M=Variants ACBP=A9
 0001:000004F4 00000006 C=CODE     S=.text    G=(none)   M=VarUtils ACBP=A9
 0001:000004FC 00000196 C=CODE     S=.text    G=(none)   M=Classes  ACBP=A9
 0001:00000694 0000048E C=CODE     S=.text    G=(none)   M=Controls ACBP=A9
 0001:00000B24 00000006 C=CODE     S=.text    G=(none)   M=ActnList ACBP=A9
 0001:00000B2C 0000001E C=CODE     S=.text    G=(none)   M=ImgList  ACBP=A9
 0001:00000B4C 0000002F C=CODE     S=.text    G=(none)   M=CommCtrl ACBP=A9
 0001:00000B7C 00000086 C=CODE     S=.text    G=(none)   M=Graphics ACBP=A9
 0001:00000C04 00000006 C=CODE     S=.text    G=(none)   M=Registry ACBP=A9
 0001:00000C0C 00000006 C=CODE     S=.text    G=(none)   M=IniFiles ACBP=A9
 0001:00000C14 00000006 C=CODE     S=.text    G=(none)   M=Themes   ACBP=A9
 0001:00000C1C 000000AE C=CODE     S=.text    G=(none)   M=Menus    ACBP=A9
 0001:00000CCC 00000006 C=CODE     S=.text    G=(none)   M=UxTheme  ACBP=A9
 0001:00000CD4 00000006 C=CODE     S=.text    G=(none)   M=MultiMon ACBP=A9
 0001:00000CDC 00000006 C=CODE     S=.text    G=(none)   M=DwmApi   ACBP=A9
 0001:00000CE4 00000016 C=CODE     S=.text    G=(none)   M=Forms    ACBP=A9
 0001:00000CFC 00000006 C=CODE     S=.text    G=(none)   M=HelpIntfs ACBP=A9
 0001:00000D04 00000006 C=CODE     S=.text    G=(none)   M=Dialogs  ACBP=A9
 0001:00000D0C 00000386 C=CODE     S=.text    G=(none)   M=StdCtrls ACBP=A9
 0001:00001094 00000006 C=CODE     S=.text    G=(none)   M=Printers ACBP=A9
 0001:0000109C 00000086 C=CODE     S=.text    G=(none)   M=ExtCtrls ACBP=A9
 0001:00001124 00000006 C=CODE     S=.text    G=(none)   M=GraphUtil ACBP=A9
 0001:0000112C 00000006 C=CODE     S=.text    G=(none)   M=Clipbrd  ACBP=A9
 0001:00001134 00000006 C=CODE     S=.text    G=(none)   M=FlatSB   ACBP=A9
 0001:0000113C 00000046 C=CODE     S=.text    G=(none)   M=CheckLst ACBP=A9
 0001:00001184 0000005E C=CODE     S=.text    G=(none)   M=Grids    ACBP=A9
 0001:000011E4 0000004E C=CODE     S=.text    G=(none)   M=Buttons  ACBP=A9
 0001:00001234 0000032E C=CODE     S=.text    G=(none)   M=ComCtrls ACBP=A9
 0001:00001564 00000006 C=CODE     S=.text    G=(none)   M=ExtActns ACBP=A9
 0001:0000156C 00000006 C=CODE     S=.text    G=(none)   M=ExtDlgs  ACBP=A9
 0001:00001574 00000006 C=CODE     S=.text    G=(none)   M=Mapi     ACBP=A9
 0001:0000157C 00000006 C=CODE     S=.text    G=(none)   M=VAUtils  ACBP=A9
 0001:00001584 00000006 C=CODE     S=.text    G=(none)   M=ComObj   ACBP=A9
 0001:0000158C 000000B6 C=CODE     S=.text    G=(none)   M=DesignEditors ACBP=A9
 0001:00001644 00000006 C=CODE     S=.text    G=(none)   M=DesignIntf ACBP=A9
 0001:0000164C 00000006 C=CODE     S=.text    G=(none)   M=ToolsAPI ACBP=A9
 0001:00001654 00000006 C=CODE     S=.text    G=(none)   M=XMLIntf  ACBP=A9
 0001:0000165C 00000006 C=CODE     S=.text    G=(none)   M=xmldom   ACBP=A9
 0001:00001664 00000006 C=CODE     S=.text    G=(none)   M=msxmldom ACBP=A9
 0001:0000166C 00000006 C=CODE     S=.text    G=(none)   M=DockForm ACBP=A9
 0001:00001674 00000006 C=CODE     S=.text    G=(none)   M=IDEMessages ACBP=A9
 0001:0000167C 00000006 C=CODE     S=.text    G=(none)   M=DeskForm ACBP=A9
 0001:00001684 00000006 C=CODE     S=.text    G=(none)   M=BaseDock ACBP=A9
 0001:0000168C 00000006 C=CODE     S=.text    G=(none)   M=PercentageDockTree ACBP=A9
 0001:00001694 00000006 C=CODE     S=.text    G=(none)   M=CaptionedDockTree ACBP=A9
 0001:0000169C 00000006 C=CODE     S=.text    G=(none)   M=DockTabSet ACBP=A9
 0001:000016A4 00000006 C=CODE     S=.text    G=(none)   M=Tabs     ACBP=A9
 0001:000016AC 00000006 C=CODE     S=.text    G=(none)   M=DeskUtil ACBP=A9
 0001:000016B4 00000006 C=CODE     S=.text    G=(none)   M=ActnMan  ACBP=A9
 0001:000016BC 00000006 C=CODE     S=.text    G=(none)   M=ActnMenus ACBP=A9
 0001:000016C4 00000006 C=CODE     S=.text    G=(none)   M=XPStyleActnCtrls ACBP=A9
 0001:000016CC 00000006 C=CODE     S=.text    G=(none)   M=Proxies  ACBP=A9
 0001:000016D4 000001C3 C=CODE     S=.text    G=(none)   M=SysInit  ACBP=A9
 0001:00001898 00011CCB C=CODE     S=.text    G=(none)   M=ORCtrls  ACBP=A9
 0001:00013564 000006E2 C=CODE     S=.text    G=(none)   M=ORCtrlsDsgn ACBP=A9
 0001:00013C48 0000039F C=CODE     S=.text    G=(none)   M=.ORCtrlLib2006 ACBP=A9
 0002:00000000 00000006 C=ICODE    S=.itext   G=(none)   M=System   ACBP=A9
 0002:00000008 00000006 C=ICODE    S=.itext   G=(none)   M=TypInfo  ACBP=A9
 0002:00000010 00000006 C=ICODE    S=.itext   G=(none)   M=SysUtils ACBP=A9
 0002:00000018 00000011 C=ICODE    S=.itext   G=(none)   M=Windows  ACBP=A9
 0002:0000002C 00000006 C=ICODE    S=.itext   G=(none)   M=Variants ACBP=A9
 0002:00000034 00000006 C=ICODE    S=.itext   G=(none)   M=VarUtils ACBP=A9
 0002:0000003C 00000006 C=ICODE    S=.itext   G=(none)   M=Classes  ACBP=A9
 0002:00000044 00000006 C=ICODE    S=.itext   G=(none)   M=Controls ACBP=A9
 0002:0000004C 00000006 C=ICODE    S=.itext   G=(none)   M=ActnList ACBP=A9
 0002:00000054 00000006 C=ICODE    S=.itext   G=(none)   M=Graphics ACBP=A9
 0002:0000005C 00000006 C=ICODE    S=.itext   G=(none)   M=Registry ACBP=A9
 0002:00000064 00000006 C=ICODE    S=.itext   G=(none)   M=IniFiles ACBP=A9
 0002:0000006C 00000006 C=ICODE    S=.itext   G=(none)   M=Themes   ACBP=A9
 0002:00000074 00000006 C=ICODE    S=.itext   G=(none)   M=Menus    ACBP=A9
 0002:0000007C 00000006 C=ICODE    S=.itext   G=(none)   M=UxTheme  ACBP=A9
 0002:00000084 00000006 C=ICODE    S=.itext   G=(none)   M=MultiMon ACBP=A9
 0002:0000008C 00000006 C=ICODE    S=.itext   G=(none)   M=DwmApi   ACBP=A9
 0002:00000094 00000006 C=ICODE    S=.itext   G=(none)   M=Forms    ACBP=A9
 0002:0000009C 00000006 C=ICODE    S=.itext   G=(none)   M=HelpIntfs ACBP=A9
 0002:000000A4 00000006 C=ICODE    S=.itext   G=(none)   M=Dialogs  ACBP=A9
 0002:000000AC 00000006 C=ICODE    S=.itext   G=(none)   M=Printers ACBP=A9
 0002:000000B4 00000006 C=ICODE    S=.itext   G=(none)   M=ExtCtrls ACBP=A9
 0002:000000BC 00000006 C=ICODE    S=.itext   G=(none)   M=GraphUtil ACBP=A9
 0002:000000C4 00000006 C=ICODE    S=.itext   G=(none)   M=Clipbrd  ACBP=A9
 0002:000000CC 00000006 C=ICODE    S=.itext   G=(none)   M=FlatSB   ACBP=A9
 0002:000000D4 00000006 C=ICODE    S=.itext   G=(none)   M=CheckLst ACBP=A9
 0002:000000DC 00000006 C=ICODE    S=.itext   G=(none)   M=Buttons  ACBP=A9
 0002:000000E4 00000006 C=ICODE    S=.itext   G=(none)   M=ComCtrls ACBP=A9
 0002:000000EC 00000006 C=ICODE    S=.itext   G=(none)   M=ExtActns ACBP=A9
 0002:000000F4 00000006 C=ICODE    S=.itext   G=(none)   M=ExtDlgs  ACBP=A9
 0002:000000FC 00000006 C=ICODE    S=.itext   G=(none)   M=Mapi     ACBP=A9
 0002:00000104 00000006 C=ICODE    S=.itext   G=(none)   M=VAUtils  ACBP=A9
 0002:0000010C 00000006 C=ICODE    S=.itext   G=(none)   M=ComObj   ACBP=A9
 0002:00000114 00000006 C=ICODE    S=.itext   G=(none)   M=DesignEditors ACBP=A9
 0002:0000011C 00000006 C=ICODE    S=.itext   G=(none)   M=ToolsAPI ACBP=A9
 0002:00000124 00000006 C=ICODE    S=.itext   G=(none)   M=XMLIntf  ACBP=A9
 0002:0000012C 00000006 C=ICODE    S=.itext   G=(none)   M=xmldom   ACBP=A9
 0002:00000134 00000006 C=ICODE    S=.itext   G=(none)   M=msxmldom ACBP=A9
 0002:0000013C 00000006 C=ICODE    S=.itext   G=(none)   M=DockForm ACBP=A9
 0002:00000144 00000006 C=ICODE    S=.itext   G=(none)   M=IDEMessages ACBP=A9
 0002:0000014C 00000006 C=ICODE    S=.itext   G=(none)   M=DeskForm ACBP=A9
 0002:00000154 00000006 C=ICODE    S=.itext   G=(none)   M=BaseDock ACBP=A9
 0002:0000015C 00000006 C=ICODE    S=.itext   G=(none)   M=PercentageDockTree ACBP=A9
 0002:00000164 00000006 C=ICODE    S=.itext   G=(none)   M=CaptionedDockTree ACBP=A9
 0002:0000016C 00000006 C=ICODE    S=.itext   G=(none)   M=DockTabSet ACBP=A9
 0002:00000174 00000006 C=ICODE    S=.itext   G=(none)   M=Tabs     ACBP=A9
 0002:0000017C 00000006 C=ICODE    S=.itext   G=(none)   M=DeskUtil ACBP=A9
 0002:00000184 00000006 C=ICODE    S=.itext   G=(none)   M=ActnMan  ACBP=A9
 0002:0000018C 00000006 C=ICODE    S=.itext   G=(none)   M=ActnMenus ACBP=A9
 0002:00000194 00000006 C=ICODE    S=.itext   G=(none)   M=XPStyleActnCtrls ACBP=A9
 0002:0000019C 00000006 C=ICODE    S=.itext   G=(none)   M=Proxies  ACBP=A9
 0002:000001A4 0000005E C=ICODE    S=.itext   G=(none)   M=ORCtrls  ACBP=A9
 0002:00000204 00000008 C=ICODE    S=.itext   G=(none)   M=ORCtrlsDsgn ACBP=A9
 0002:0000020C 00000005 C=ICODE    S=.itext   G=(none)   M=.ORCtrlLib2006 ACBP=A9
 0003:00000000 00000030 C=DATA     S=.data    G=DGROUP   M=SysInit  ACBP=A9
 0003:00000030 00000248 C=DATA     S=.data    G=DGROUP   M=ORCtrls  ACBP=A9
 0004:00000000 00000008 C=BSS      S=.bss     G=DGROUP   M=Windows  ACBP=A9
 0004:00000008 0000000C C=BSS      S=.bss     G=DGROUP   M=SysInit  ACBP=A9
 0004:00000014 00000099 C=BSS      S=.bss     G=DGROUP   M=ORCtrls  ACBP=A9
 0004:000000B0 00000004 C=BSS      S=.bss     G=DGROUP   M=ORCtrlsDsgn ACBP=A9


  Address             Publics by Name

 0002:0000020C       .ORCtrlLib2006..ORCtrlLib2006
 0001:00013FC8       .ORCtrlLib2006.@GetPackageInfoTable
 0001:00013FD0       .ORCtrlLib2006.@PackageLoad
 0001:00013FDC       .ORCtrlLib2006.@PackageUnload
 0001:00000B4C       CommCtrl.TreeView_GetItem
 0001:00000B64       CommCtrl.TreeView_SetItem
 0004:00000014       ORCtrls..03
 0001:000053EC       ORCtrls..TCaptionCheckListBox
 0001:00005D04       ORCtrls..TCaptionComboBox
 0001:00005874       ORCtrls..TCaptionEdit
 0001:00005148       ORCtrls..TCaptionListBox
 0001:00005F58       ORCtrls..TCaptionListView
 0001:00005658       ORCtrls..TCaptionMemo
 0001:00005AA8       ORCtrls..TCaptionRichEdit
 0001:000061B8       ORCtrls..TCaptionStringGrid
 0001:00003E5C       ORCtrls..TCaptionTreeView
 0001:000063A0       ORCtrls..TItemTip
 0001:00004DE8       ORCtrls..TKeyClickPanel
 0001:00004F50       ORCtrls..TKeyClickRadioGroup
 0001:0000389C       ORCtrls..TORAlignButton
 0001:00003BF0       ORCtrls..TORAlignEdit
 0001:00003A8C       ORCtrls..TORAlignSpeedButton
 0001:000032AC       ORCtrls..TORAutoPanel
 0001:0000441C       ORCtrls..TORCBImageIndexes
 0001:000046AC       ORCtrls..TORCheckBox
 0001:0000283C       ORCtrls..TORComboBox
 0001:000025DC       ORCtrls..TORComboEdit
 0001:00002474       ORCtrls..TORComboPanelEdit
 0001:000022C8       ORCtrls..TORDropPanel
 0001:00001D28       ORCtrls..TORListBox
 0001:00004A64       ORCtrls..TORListView
 0001:00004D0C       ORCtrls..TORMenuItem
 0001:00003414       ORCtrls..TOROffsetLabel
 0001:00004C34       ORCtrls..TORPopupMenu
 0001:00001910       ORCtrls..TORStrings
 0001:00004038       ORCtrls..TORTreeNode
 0001:0000412C       ORCtrls..TORTreeView
 0001:000064F8       ORCtrls..TSizeRatio
 0001:00006B78       ORCtrls.AddItemTipRef
 0003:00000030       ORCtrls.ALPHA_DISTRIBUTION
 0003:00000204       ORCtrls.BlackCheckBoxImageResNames
 0003:00000250       ORCtrls.BlackComboBoxImages
 0003:00000258       ORCtrls.ButtonAlignment
 0003:0000026C       ORCtrls.ButtonLayout
 0003:00000264       ORCtrls.ButtonWordWrap
 0001:00010250       ORCtrls.CalcShortName
 0003:000001C4       ORCtrls.CheckBoxImageResNames
 0001:0000B834       ORCtrls.ClearLong
 0001:00006574       ORCtrls.ClientWidthOfList
 0003:00000248       ORCtrls.ComboBoxImages
 0001:000075AC       ORCtrls.DestroyORCBBitmaps
 0001:0000CB48       ORCtrls.DropDownPanelClosed
 0001:0000CB1C       ORCtrls.DropDownPanelOpened
 0001:00012280       ORCtrls.EnableCtrl
 0001:000134F4       ORCtrls.Finalization
 0001:000066BC       ORCtrls.FontHeightPixel
 0001:000065B8       ORCtrls.FontWidthPixel
 0001:000074E8       ORCtrls.GetORCBBitmap
 0001:0001312C       ORCtrls.GoodNotifyWinEvent
 0001:00006700       ORCtrls.HigherOf
 0004:00000028       ORCtrls.HintArray
 0001:000068D0       ORCtrls.IntArrayToString
 0001:00013294       ORCtrls.IsAMouseButtonDown
 0001:00006B44       ORCtrls.ItemTipKeyHook
 0001:0000670C       ORCtrls.LowerOf
 0004:0000002C       ORCtrls.ORCBImages
 0002:000001A4       ORCtrls.ORCtrls
 0001:00006718       ORCtrls.Piece
 0001:00006BB0       ORCtrls.RemoveItemTipRef
 0001:00010D94       ORCtrls.RStr
 0001:000067A8       ORCtrls.SetPiece
 0001:00006B0C       ORCtrls.StringBetween
 0001:000069A0       ORCtrls.StringToIntArray
 0001:00012C40       ORCtrls.TCaptionCheckListBox.GetCaption
 0001:00012C6C       ORCtrls.TCaptionCheckListBox.GetDynamicProperty
 0001:00012C90       ORCtrls.TCaptionCheckListBox.SetCaption
 0001:00012D14       ORCtrls.TCaptionCheckListBox.SupportsDynamicProperty
 0001:00012FD8       ORCtrls.TCaptionComboBox.GetCaption
 0001:00013004       ORCtrls.TCaptionComboBox.GetDynamicProperty
 0001:00013028       ORCtrls.TCaptionComboBox.SetCaption
 0001:000130AC       ORCtrls.TCaptionComboBox.SupportsDynamicProperty
 0001:00012DF8       ORCtrls.TCaptionEdit.GetCaption
 0001:00012E24       ORCtrls.TCaptionEdit.GetDynamicProperty
 0001:00012E48       ORCtrls.TCaptionEdit.SetCaption
 0001:00012ECC       ORCtrls.TCaptionEdit.SupportsDynamicProperty
 0001:00012810       ORCtrls.TCaptionListBox.DoEnter
 0001:00012834       ORCtrls.TCaptionListBox.GetCaption
 0001:00012860       ORCtrls.TCaptionListBox.GetDynamicProperty
 0001:000128C0       ORCtrls.TCaptionListBox.MoveFocusDown
 0001:00012884       ORCtrls.TCaptionListBox.MoveFocusUp
 0001:00012914       ORCtrls.TCaptionListBox.SetCaption
 0001:00012998       ORCtrls.TCaptionListBox.SupportsDynamicProperty
 0001:000129A0       ORCtrls.TCaptionListBox.WMKeyDown
 0001:00012A4C       ORCtrls.TCaptionListBox.WMMouseMove
 0001:00012B0C       ORCtrls.TCaptionListBox.WMRButtonUp
 0001:000134C8       ORCtrls.TCaptionListView.GetDynamicProperty
 0001:000134EC       ORCtrls.TCaptionListView.SupportsDynamicProperty
 0001:00012D1C       ORCtrls.TCaptionMemo.GetCaption
 0001:00012D48       ORCtrls.TCaptionMemo.GetDynamicProperty
 0001:00012D6C       ORCtrls.TCaptionMemo.SetCaption
 0001:00012DF0       ORCtrls.TCaptionMemo.SupportsDynamicProperty
 0001:00012ED4       ORCtrls.TCaptionRichEdit.GetDynamicProperty
 0001:00012EFC       ORCtrls.TCaptionRichEdit.SupportsDynamicProperty
 0001:00013134       ORCtrls.TCaptionStringGrid.ColRowToIndex
 0001:00013184       ORCtrls.TCaptionStringGrid.GetDynamicProperty
 0001:000131AC       ORCtrls.TCaptionStringGrid.IndexToColRow
 0001:00013210       ORCtrls.TCaptionStringGrid.KeyUp
 0001:0001328C       ORCtrls.TCaptionStringGrid.SupportsDynamicProperty
 0001:00012F04       ORCtrls.TCaptionTreeView.GetCaption
 0001:00012F1C       ORCtrls.TCaptionTreeView.GetDynamicProperty
 0001:00012F40       ORCtrls.TCaptionTreeView.SetCaption
 0001:00012FD0       ORCtrls.TCaptionTreeView.SupportsDynamicProperty
 0001:00006BE0       ORCtrls.TItemTip.Create
 0001:00006C70       ORCtrls.TItemTip.CreateParams
 0001:00006C34       ORCtrls.TItemTip.Destroy
 0001:00006DC8       ORCtrls.TItemTip.GetTabSettings
 0001:00006D84       ORCtrls.TItemTip.Hide
 0001:00006C9C       ORCtrls.TItemTip.Paint
 0001:0000719C       ORCtrls.TItemTip.Show
 0001:00006EF4       ORCtrls.TItemTip.UpdateText
 0001:000126E4       ORCtrls.TKeyClickPanel.KeyDown
 0001:00012708       ORCtrls.TKeyClickRadioGroup.Click
 0001:00012740       ORCtrls.TKeyClickRadioGroup.Create
 0001:000127A0       ORCtrls.TKeyClickRadioGroup.KeyDown
 0001:0000FE64       ORCtrls.TORAlignButton.Create
 0001:0000FEB4       ORCtrls.TORAlignButton.CreateParams
 0001:0000FEFC       ORCtrls.TORAlignButton.SetAlignment
 0001:0000FF14       ORCtrls.TORAlignButton.SetLayout
 0001:0000FF2C       ORCtrls.TORAlignButton.SetWordWrap
 0001:000130B4       ORCtrls.TORAlignSpeedButton.Paint
 0001:0000F870       ORCtrls.TORAutoPanel.BuildSizes
 0001:0000F7F8       ORCtrls.TORAutoPanel.Destroy
 0001:0000F99C       ORCtrls.TORAutoPanel.DoResize
 0001:0000F968       ORCtrls.TORAutoPanel.Loaded
 0001:0000FB44       ORCtrls.TORAutoPanel.Resize
 0001:00010C9C       ORCtrls.TORCBImageIndexes.Create
 0001:00010D20       ORCtrls.TORCBImageIndexes.Destroy
 0001:00010DD0       ORCtrls.TORCBImageIndexes.IdxString
 0001:00011014       ORCtrls.TORCBImageIndexes.ImageListChanged
 0001:00011048       ORCtrls.TORCBImageIndexes.Notification
 0001:00011078       ORCtrls.TORCBImageIndexes.SetCheckedDisabledIndex
 0001:0001108C       ORCtrls.TORCBImageIndexes.SetCheckedEnabledIndex
 0001:000110A0       ORCtrls.TORCBImageIndexes.SetGrayedDisabledIndex
 0001:000110B4       ORCtrls.TORCBImageIndexes.SetGrayedEnabledIndex
 0001:00010EB4       ORCtrls.TORCBImageIndexes.SetIdxString
 0001:00010D54       ORCtrls.TORCBImageIndexes.SetImages
 0001:000110C8       ORCtrls.TORCBImageIndexes.SetUncheckedDisabledIndex
 0001:000110DC       ORCtrls.TORCBImageIndexes.SetUncheckedEnabledIndex
 0001:00011F00       ORCtrls.TORCheckBox.AutoAdjustSize
 0001:00012384       ORCtrls.TORCheckBox.BMGetCheck
 0001:000123B0       ORCtrls.TORCheckBox.BMGetState
 0001:00011D8C       ORCtrls.TORCheckBox.BMSetCheck
 0001:00011304       ORCtrls.TORCheckBox.CMEnabledChanged
 0001:00011320       ORCtrls.TORCheckBox.CMFontChanged
 0001:0001133C       ORCtrls.TORCheckBox.CNDrawItem
 0001:00011358       ORCtrls.TORCheckBox.CNMeasureItem
 0001:000110F0       ORCtrls.TORCheckBox.Create
 0001:00011198       ORCtrls.TORCheckBox.CreateCommon
 0001:000112E8       ORCtrls.TORCheckBox.CreateParams
 0001:000111C8       ORCtrls.TORCheckBox.Destroy
 0001:00011934       ORCtrls.TORCheckBox.DrawItem
 0001:000120D4       ORCtrls.TORCheckBox.GetCaption
 0001:0001137C       ORCtrls.TORCheckBox.GetDrawData
 0001:00011210       ORCtrls.TORCheckBox.GetImageIndexes
 0001:0001122C       ORCtrls.TORCheckBox.GetImageList
 0001:0001114C       ORCtrls.TORCheckBox.ListViewCreate
 0001:0001233C       ORCtrls.TORCheckBox.Notification
 0001:00012158       ORCtrls.TORCheckBox.SetAllowAllUnchecked
 0001:00012244       ORCtrls.TORCheckBox.SetAssociate
 0001:00011EBC       ORCtrls.TORCheckBox.SetAutoSize
 0001:00011EE4       ORCtrls.TORCheckBox.SetBlackColorMode
 0001:000120EC       ORCtrls.TORCheckBox.SetCaption
 0001:00012370       ORCtrls.TORCheckBox.SetFocusOnBox
 0001:00011D28       ORCtrls.TORCheckBox.SetGrayedStyle
 0001:00012168       ORCtrls.TORCheckBox.SetGroupIndex
 0001:00011238       ORCtrls.TORCheckBox.SetImageIndexes
 0001:00011248       ORCtrls.TORCheckBox.SetImageList
 0001:00012218       ORCtrls.TORCheckBox.SetParent
 0001:00012230       ORCtrls.TORCheckBox.SetRadioStyle
 0001:00011E94       ORCtrls.TORCheckBox.SetWordWrap
 0001:00012198       ORCtrls.TORCheckBox.SyncAllowAllUnchecked
 0001:00011258       ORCtrls.TORCheckBox.Toggle
 0001:0001231C       ORCtrls.TORCheckBox.UpdateAssociate
 0001:00011D4C       ORCtrls.TORCheckBox.WMLButtonDblClk
 0001:00011D64       ORCtrls.TORCheckBox.WMSize
 0001:0000E9D0       ORCtrls.TORComboBox.AddReference
 0001:0000D3AC       ORCtrls.TORComboBox.AdjustSizeOfSelf
 0001:0000F6D8       ORCtrls.TORComboBox.CheckBoxSelected
 0001:0000EA34       ORCtrls.TORComboBox.Clear
 0001:0000D66C       ORCtrls.TORComboBox.ClearDropDownStatus
 0001:0000EA5C       ORCtrls.TORComboBox.ClearTop
 0001:0000D2EC       ORCtrls.TORComboBox.CMFontChanged
 0001:0000D118       ORCtrls.TORComboBox.Create
 0001:0000D684       ORCtrls.TORComboBox.Destroy
 0001:0000D6B4       ORCtrls.TORComboBox.DoEnter
 0001:0000D70C       ORCtrls.TORComboBox.DoExit
 0001:0000D52C       ORCtrls.TORComboBox.DropButtonDown
 0001:0000D55C       ORCtrls.TORComboBox.DropButtonUp
 0001:0000D58C       ORCtrls.TORComboBox.DropDownStatusChanged
 0001:0000F330       ORCtrls.TORComboBox.DropPanelBtnPressed
 0001:0000D398       ORCtrls.TORComboBox.EditControl
 0001:0000EA6C       ORCtrls.TORComboBox.ForDataUse
 0001:0000D808       ORCtrls.TORComboBox.FwdChange
 0001:0000D83C       ORCtrls.TORComboBox.FwdChangeDelayed
 0001:0000DB4C       ORCtrls.TORComboBox.FwdClick
 0001:0000DCA0       ORCtrls.TORComboBox.FwdDblClick
 0001:0000DCC4       ORCtrls.TORComboBox.FwdKeyDown
 0001:0000E0A0       ORCtrls.TORComboBox.FwdKeyPress
 0001:0000E110       ORCtrls.TORComboBox.FwdKeyUp
 0001:0000E17C       ORCtrls.TORComboBox.FwdMouseUp
 0001:0000E1A0       ORCtrls.TORComboBox.FwdNeedData
 0001:0000EC08       ORCtrls.TORComboBox.GetAutoSelect
 0001:0000F724       ORCtrls.TORComboBox.GetCaption
 0001:0000F740       ORCtrls.TORComboBox.GetCaseChanged
 0001:0000F0A4       ORCtrls.TORComboBox.GetCheckBoxes
 0001:0000F0B4       ORCtrls.TORComboBox.GetChecked
 0001:0000F398       ORCtrls.TORComboBox.GetCheckedString
 0001:0000F0C4       ORCtrls.TORComboBox.GetCheckEntireLine
 0001:0000EC18       ORCtrls.TORComboBox.GetColor
 0001:0000EC24       ORCtrls.TORComboBox.GetDelimiter
 0001:0000EC34       ORCtrls.TORComboBox.GetDisplayText
 0001:0000EC54       ORCtrls.TORComboBox.GetDynamicProperty
 0001:0000F548       ORCtrls.TORComboBox.GetEditBoxText
 0001:0000F500       ORCtrls.TORComboBox.GetEnabled
 0001:0000F0D4       ORCtrls.TORComboBox.GetFlatCheckBoxes
 0001:0000EDE4       ORCtrls.TORComboBox.GetHideSynonyms
 0001:0000EC88       ORCtrls.TORComboBox.GetIEN
 0001:0000EC78       ORCtrls.TORComboBox.GetItemHeight
 0001:0000ECAC       ORCtrls.TORComboBox.GetItemID
 0001:0000ECC8       ORCtrls.TORComboBox.GetItemIEN
 0001:0000ECEC       ORCtrls.TORComboBox.GetItemIndex
 0001:0000ED10       ORCtrls.TORComboBox.GetItemTipColor
 0001:0000ED00       ORCtrls.TORComboBox.GetItemTipEnable
 0001:0000ED20       ORCtrls.TORComboBox.GetLongList
 0001:0000F760       ORCtrls.TORComboBox.GetLookupPiece
 0001:0000ED30       ORCtrls.TORComboBox.GetMaxLength
 0001:0000F70C       ORCtrls.TORComboBox.GetMItems
 0001:0000F4C8       ORCtrls.TORComboBox.GetOnSynonymCheck
 0001:0000ED40       ORCtrls.TORComboBox.GetPieces
 0001:0000ED5C       ORCtrls.TORComboBox.GetReference
 0001:0000ED7C       ORCtrls.TORComboBox.GetSelLength
 0001:0000ED90       ORCtrls.TORComboBox.GetSelStart
 0001:0000EDA4       ORCtrls.TORComboBox.GetSelText
 0001:0000EDC4       ORCtrls.TORComboBox.GetShortCount
 0001:0000EDD4       ORCtrls.TORComboBox.GetSorted
 0001:0000EDF4       ORCtrls.TORComboBox.GetSynonymChars
 0001:0000EE90       ORCtrls.TORComboBox.GetTabPosInPixels
 0001:0000EE74       ORCtrls.TORComboBox.GetTabPositions
 0001:0000EEA0       ORCtrls.TORComboBox.GetText
 0001:0000EACC       ORCtrls.TORComboBox.IndexOfReference
 0001:0000EA7C       ORCtrls.TORComboBox.InitLongList
 0001:0000EB2C       ORCtrls.TORComboBox.InsertReference
 0001:0000EB94       ORCtrls.TORComboBox.InsertSeparator
 0001:0000EBA4       ORCtrls.TORComboBox.Invalidate
 0001:0000D754       ORCtrls.TORComboBox.LoadComboBoxImage
 0001:0000D7EC       ORCtrls.TORComboBox.Loaded
 0001:0000EEBC       ORCtrls.TORComboBox.SelectAll
 0001:0000E70C       ORCtrls.TORComboBox.SelectByID
 0001:0000E6E0       ORCtrls.TORComboBox.SelectByIEN
 0001:0000EECC       ORCtrls.TORComboBox.SetAutoSelect
 0001:0000EEDC       ORCtrls.TORComboBox.SetBlackColorMode
 0001:0000F714       ORCtrls.TORComboBox.SetCaption
 0001:0000F750       ORCtrls.TORComboBox.SetCaseChanged
 0001:0000F3C4       ORCtrls.TORComboBox.SetCheckBoxEditColor
 0001:0000F0E4       ORCtrls.TORComboBox.SetCheckBoxes
 0001:0000F2D8       ORCtrls.TORComboBox.SetChecked
 0001:0000F3B4       ORCtrls.TORComboBox.SetCheckedString
 0001:0000F310       ORCtrls.TORComboBox.SetCheckEntireLine
 0001:0000EF08       ORCtrls.TORComboBox.SetColor
 0001:0000EF40       ORCtrls.TORComboBox.SetDelimiter
 0001:0000E218       ORCtrls.TORComboBox.SetDropDownCount
 0001:0000E224       ORCtrls.TORComboBox.SetDroppedDown
 0001:0000E488       ORCtrls.TORComboBox.SetEditRect
 0001:0000E558       ORCtrls.TORComboBox.SetEditText
 0001:0000F50C       ORCtrls.TORComboBox.SetEnabled
 0001:0000E730       ORCtrls.TORComboBox.SetExactByIEN
 0001:0000F320       ORCtrls.TORComboBox.SetFlatCheckBoxes
 0001:0000EE14       ORCtrls.TORComboBox.SetHideSynonyms
 0001:0000EF50       ORCtrls.TORComboBox.SetItemHeight
 0001:0000E5FC       ORCtrls.TORComboBox.SetItemIndex
 0001:0000F090       ORCtrls.TORComboBox.SetItems
 0001:0000EF70       ORCtrls.TORComboBox.SetItemTipColor
 0001:0000EF60       ORCtrls.TORComboBox.SetItemTipEnable
 0001:0000F3F8       ORCtrls.TORComboBox.SetListItemsOnly
 0001:0000EF80       ORCtrls.TORComboBox.SetLongList
 0001:0000F770       ORCtrls.TORComboBox.SetLookupPiece
 0001:0000EF90       ORCtrls.TORComboBox.SetMaxLength
 0001:000132CC       ORCtrls.TORComboBox.SetNumForMatch
 0001:0000F418       ORCtrls.TORComboBox.SetOnCheckedText
 0001:0000F4E0       ORCtrls.TORComboBox.SetOnSynonymCheck
 0001:0000EFA0       ORCtrls.TORComboBox.SetPieces
 0001:0000EFB0       ORCtrls.TORComboBox.SetReference
 0001:0000F010       ORCtrls.TORComboBox.SetSelLength
 0001:0000F028       ORCtrls.TORComboBox.SetSelStart
 0001:0000F040       ORCtrls.TORComboBox.SetSelText
 0001:0000F050       ORCtrls.TORComboBox.SetSorted
 0001:0000E75C       ORCtrls.TORComboBox.SetStyle
 0001:0000EE24       ORCtrls.TORComboBox.SetSynonymChars
 0001:0000F070       ORCtrls.TORComboBox.SetTabPosInPixels
 0001:0000F060       ORCtrls.TORComboBox.SetTabPositions
 0001:0000F480       ORCtrls.TORComboBox.SetTemplateField
 0001:0000F080       ORCtrls.TORComboBox.SetText
 0001:0001344C       ORCtrls.TORComboBox.SetTextAutoComplete
 0001:000132F4       ORCtrls.TORComboBox.SetUniqueAutoComplete
 0001:0000E92C       ORCtrls.TORComboBox.StartKeyTimer
 0001:0000E99C       ORCtrls.TORComboBox.StopKeyTimer
 0001:0000E9C8       ORCtrls.TORComboBox.SupportsDynamicProperty
 0001:0000D6DC       ORCtrls.TORComboBox.UMGotFocus
 0001:0000F658       ORCtrls.TORComboBox.UpdateCheckEditBoxText
 0001:0000D2BC       ORCtrls.TORComboBox.WMDestroy
 0001:0000D304       ORCtrls.TORComboBox.WMMove
 0001:0000D320       ORCtrls.TORComboBox.WMSize
 0001:0000D338       ORCtrls.TORComboBox.WMTimer
 0001:0000D008       ORCtrls.TORComboEdit.CreateParams
 0001:0000D040       ORCtrls.TORComboEdit.WMKillFocus
 0001:0000D0BC       ORCtrls.TORComboEdit.WMSetFocus
 0001:000125E4       ORCtrls.TORComboPanelEdit.Destroy
 0001:0001261C       ORCtrls.TORComboPanelEdit.Paint
 0001:0000CB78       ORCtrls.TORDropPanel.BtnClicked
 0001:0000CBB0       ORCtrls.TORDropPanel.Create
 0001:0000CC28       ORCtrls.TORDropPanel.CreateParams
 0001:0000CC68       ORCtrls.TORDropPanel.GetButton
 0001:0000CD18       ORCtrls.TORDropPanel.ResetButtons
 0001:0000CD4C       ORCtrls.TORDropPanel.Resize
 0001:0000CDE4       ORCtrls.TORDropPanel.UpdateButtons
 0001:0000CF68       ORCtrls.TORDropPanel.WMActivateApp
 0001:0000A808       ORCtrls.TORListBox.AddReference
 0001:0000B16C       ORCtrls.TORListBox.AdjustScrollBar
 0001:0000CA3C       ORCtrls.TORListBox.Clear
 0001:0000B7D0       ORCtrls.TORListBox.ClearTop
 0001:00009034       ORCtrls.TORListBox.Click
 0001:0000874C       ORCtrls.TORListBox.CMFontChanged
 0001:00008FD4       ORCtrls.TORListBox.CMHintShow
 0001:00009940       ORCtrls.TORListBox.CNDrawItem
 0001:00007D60       ORCtrls.TORListBox.Create
 0001:00007EB4       ORCtrls.TORListBox.CreateParams
 0001:0000B208       ORCtrls.TORListBox.CreateScrollBar
 0001:00007ECC       ORCtrls.TORListBox.CreateWnd
 0001:00007E60       ORCtrls.TORListBox.Destroy
 0001:00009148       ORCtrls.TORListBox.DestroyItems
 0001:00007F58       ORCtrls.TORListBox.DestroyWnd
 0001:00009050       ORCtrls.TORListBox.DoChange
 0001:000090BC       ORCtrls.TORListBox.DoEnter
 0001:000090FC       ORCtrls.TORListBox.DoExit
 0001:00009964       ORCtrls.TORListBox.DrawItem
 0001:0000B2DC       ORCtrls.TORListBox.ForDataUse
 0001:0000B2B8       ORCtrls.TORListBox.FreeScrollBar
 0001:0000CB00       ORCtrls.TORListBox.GetCaption
 0001:0000C6B0       ORCtrls.TORListBox.GetChecked
 0001:0000C78C       ORCtrls.TORListBox.GetCheckedState
 0001:0000C87C       ORCtrls.TORListBox.GetCheckedString
 0001:00008168       ORCtrls.TORListBox.GetDisplayText
 0001:000081C4       ORCtrls.TORListBox.GetDynamicProperty
 0001:0000A274       ORCtrls.TORListBox.GetIEN
 0001:00009DD0       ORCtrls.TORListBox.GetIndexFromY
 0001:0000A538       ORCtrls.TORListBox.GetItemID
 0001:0000A324       ORCtrls.TORListBox.GetItemIEN
 0001:0000C9C0       ORCtrls.TORListBox.GetMItems
 0001:0000C850       ORCtrls.TORListBox.GetMultiSelect
 0001:0000AED8       ORCtrls.TORListBox.GetPieces
 0001:0000A698       ORCtrls.TORListBox.GetReference
 0001:0000C1F8       ORCtrls.TORListBox.GetStringIndex
 0001:0000AE8C       ORCtrls.TORListBox.GetStyle
 0001:0000A99C       ORCtrls.TORListBox.GetTabPositions
 0001:0000A8EC       ORCtrls.TORListBox.IndexOfReference
 0001:0000B594       ORCtrls.TORListBox.InitLongList
 0001:0000A878       ORCtrls.TORListBox.InsertReference
 0001:0000B728       ORCtrls.TORListBox.InsertSeparator
 0001:00008074       ORCtrls.TORListBox.IsSynonym
 0001:000092B4       ORCtrls.TORListBox.KeyPress
 0001:00008418       ORCtrls.TORListBox.LBAddString
 0001:00008610       ORCtrls.TORListBox.LBDeleteString
 0001:000081E8       ORCtrls.TORListBox.LBGetItemData
 0001:000082A8       ORCtrls.TORListBox.LBGetText
 0001:00008374       ORCtrls.TORListBox.LBGetTextLen
 0001:00008504       ORCtrls.TORListBox.LBInsertString
 0001:00008694       ORCtrls.TORListBox.LBResetContent
 0001:00008730       ORCtrls.TORListBox.LBSetCurSel
 0001:0000821C       ORCtrls.TORListBox.LBSetItemData
 0001:00007F24       ORCtrls.TORListBox.Loaded
 0001:00009870       ORCtrls.TORListBox.MeasureItem
 0001:000092E8       ORCtrls.TORListBox.MouseDown
 0001:00009654       ORCtrls.TORListBox.MouseMove
 0001:0000B924       ORCtrls.TORListBox.NeedData
 0001:0000BC40       ORCtrls.TORListBox.PositionThumb
 0001:0000AF1C       ORCtrls.TORListBox.ResetItems
 0001:0000BCF0       ORCtrls.TORListBox.ScrollTo
 0001:0000A5D4       ORCtrls.TORListBox.SelectByID
 0001:0000A3D4       ORCtrls.TORListBox.SelectByIEN
 0001:0000C340       ORCtrls.TORListBox.SelectString
 0001:0000CA58       ORCtrls.TORListBox.SetBlackColorMode
 0001:0000CA60       ORCtrls.TORListBox.SetCaption
 0001:0000C644       ORCtrls.TORListBox.SetCheckBoxes
 0001:0000C6F8       ORCtrls.TORListBox.SetChecked
 0001:0000C7C8       ORCtrls.TORListBox.SetCheckedState
 0001:0000C924       ORCtrls.TORListBox.SetCheckedString
 0001:0000AEC8       ORCtrls.TORListBox.SetDelimiter
 0001:0000A438       ORCtrls.TORListBox.SetExactByIEN
 0001:0000C694       ORCtrls.TORListBox.SetFlatCheckBoxes
 0001:00009E64       ORCtrls.TORListBox.SetFocusIndex
 0001:0000AD34       ORCtrls.TORListBox.SetHideSynonyms
 0001:0000936C       ORCtrls.TORListBox.SetHintProperties
 0001:0000B134       ORCtrls.TORListBox.SetLongList
 0001:0000C9F8       ORCtrls.TORListBox.SetMItems
 0001:0000C858       ORCtrls.TORListBox.SetMultiSelect
 0001:0000AEF8       ORCtrls.TORListBox.SetPieces
 0001:0000A734       ORCtrls.TORListBox.SetReference
 0001:0000AE94       ORCtrls.TORListBox.SetStyle
 0001:0000ADF8       ORCtrls.TORListBox.SetSynonymChars
 0001:0000AB84       ORCtrls.TORListBox.SetTabPosInPixels
 0001:0000A9D8       ORCtrls.TORListBox.SetTabPositions
 0001:0000AB9C       ORCtrls.TORListBox.SetTabStops
 0001:0000AD2C       ORCtrls.TORListBox.SupportsDynamicProperty
 0001:00007F78       ORCtrls.TORListBox.TextToShow
 0001:000091C0       ORCtrls.TORListBox.ToggleCheckBox
 0001:0000A13C       ORCtrls.TORListBox.UMShowTip
 0001:000132FC       ORCtrls.TORListBox.VerifyUnique
 0001:00008F14       ORCtrls.TORListBox.WMCancelMode
 0001:00009914       ORCtrls.TORListBox.WMDestroy
 0001:00008784       ORCtrls.TORListBox.WMKeyDown
 0001:00008D4C       ORCtrls.TORListBox.WMLButtonDblClk
 0001:000089A0       ORCtrls.TORListBox.WMLButtonDown
 0001:00008C54       ORCtrls.TORListBox.WMLButtonUp
 0001:00008F48       ORCtrls.TORListBox.WMMove
 0001:00008C9C       ORCtrls.TORListBox.WMRButtonUp
 0001:00008F68       ORCtrls.TORListBox.WMSize
 0001:00008FB0       ORCtrls.TORListBox.WMVScroll
 0001:0001247C       ORCtrls.TORListView.LVMSetColumn
 0001:00012530       ORCtrls.TORListView.LVMSetColumnWidth
 0001:000123B4       ORCtrls.TORListView.WMNotify
 0001:0000FC00       ORCtrls.TOROffsetLabel.AdjustSizeOfSelf
 0001:0000FBE8       ORCtrls.TOROffsetLabel.CMFontChanged
 0001:0000FBD0       ORCtrls.TOROffsetLabel.CMTextChanged
 0001:0000FB70       ORCtrls.TOROffsetLabel.Create
 0001:0000FCA0       ORCtrls.TOROffsetLabel.DoDrawText
 0001:0000FDDC       ORCtrls.TOROffsetLabel.GetTransparent
 0001:0000FD40       ORCtrls.TOROffsetLabel.Paint
 0001:0000FE3C       ORCtrls.TOROffsetLabel.SetHorzOffset
 0001:0000FDE8       ORCtrls.TOROffsetLabel.SetTransparent
 0001:0000FE2C       ORCtrls.TOROffsetLabel.SetVertOffset
 0001:0000FE4C       ORCtrls.TOROffsetLabel.SetWordWrap
 0001:000075E0       ORCtrls.TORStrings.Add
 0001:00007660       ORCtrls.TORStrings.Clear
 0001:00007690       ORCtrls.TORStrings.Create
 0001:000076E8       ORCtrls.TORStrings.Delete
 0001:00007720       ORCtrls.TORStrings.Destroy
 0001:00007754       ORCtrls.TORStrings.Get
 0001:0000777C       ORCtrls.TORStrings.GetCount
 0001:00007794       ORCtrls.TORStrings.GetObject
 0001:000077B4       ORCtrls.TORStrings.IndexOf
 0001:000077D4       ORCtrls.TORStrings.Insert
 0001:0000785C       ORCtrls.TORStrings.Put
 0001:000078DC       ORCtrls.TORStrings.PutObject
 0001:000078F8       ORCtrls.TORStrings.SetUpdateState
 0001:00007914       ORCtrls.TORStrings.Verify
 0001:0000FF44       ORCtrls.TORTreeNode.EnsureVisible
 0001:0000FFF4       ORCtrls.TORTreeNode.GetBold
 0001:00010030       ORCtrls.TORTreeNode.GetORTreeView
 0001:0001004C       ORCtrls.TORTreeNode.GetParent
 0001:00010068       ORCtrls.TORTreeNode.GetText
 0001:00010080       ORCtrls.TORTreeNode.SetBold
 0001:0001047C       ORCtrls.TORTreeNode.SetCaption
 0001:000100C4       ORCtrls.TORTreeNode.SetPiece
 0001:00010108       ORCtrls.TORTreeNode.SetStringData
 0001:000101B4       ORCtrls.TORTreeNode.SetText
 0001:000101C0       ORCtrls.TORTreeNode.UpdateText
 0001:0001052C       ORCtrls.TORTreeView.CNNotify
 0001:000105B8       ORCtrls.TORTreeView.Create
 0001:000105F8       ORCtrls.TORTreeView.CreateNode
 0001:00010694       ORCtrls.TORTreeView.FindPieceNode
 0001:00010634       ORCtrls.TORTreeView.FindPieceNode
 0001:0001077C       ORCtrls.TORTreeView.GetExpandedIDStr
 0001:00010A08       ORCtrls.TORTreeView.GetHorzScrollPos
 0001:00010BA0       ORCtrls.TORTreeView.GetNodeID
 0001:00010BC8       ORCtrls.TORTreeView.GetNodeID
 0001:00010A20       ORCtrls.TORTreeView.GetVertScrollPos
 0001:00010A38       ORCtrls.TORTreeView.RenameNodes
 0001:00010888       ORCtrls.TORTreeView.SetExpandedIDStr
 0001:00010878       ORCtrls.TORTreeView.SetExpandedIDStr
 0001:00010B10       ORCtrls.TORTreeView.SetHorzScrollPos
 0001:00010AF8       ORCtrls.TORTreeView.SetNodeDelim
 0001:00010B4C       ORCtrls.TORTreeView.SetNodePiece
 0001:00010C8C       ORCtrls.TORTreeView.SetShortNodeCaptions
 0001:00010B64       ORCtrls.TORTreeView.SetVertScrollPos
 0001:0000F780       ORCtrls.TSizeRatio.Create
 0003:00000244       ORCtrls.uDropPanelOpenCount
 0004:0000001C       ORCtrls.uItemTip
 0004:00000020       ORCtrls.uItemTipCount
 0004:00000018       ORCtrls.uKeyHookHandle
 0004:00000024       ORCtrls.uNewStyle
 0004:000000AC       ORCtrls.uOldShowHintsSetting
 0004:000000B0       ORCtrlsDsgn..3
 0001:00013654       ORCtrlsDsgn..TORImageIndexesElementPropertyEditor
 0001:00013564       ORCtrlsDsgn..TORImageIndexesPropertyEditor
 0001:00013C18       ORCtrlsDsgn.Finalization
 0002:00000204       ORCtrlsDsgn.ORCtrlsDsgn
 0001:00013B10       ORCtrlsDsgn.Register
 0001:000137C4       ORCtrlsDsgn.TORImageIndexesElementPropertyEditor.Create
 0001:0001384C       ORCtrlsDsgn.TORImageIndexesElementPropertyEditor.GetAttributes
 0001:00013858       ORCtrlsDsgn.TORImageIndexesElementPropertyEditor.GetName
 0001:00013994       ORCtrlsDsgn.TORImageIndexesElementPropertyEditor.GetValue
 0001:00013810       ORCtrlsDsgn.TORImageIndexesElementPropertyEditor.ParentImgIdx
 0001:00013A5C       ORCtrlsDsgn.TORImageIndexesElementPropertyEditor.SetValue
 0001:00013760       ORCtrlsDsgn.TORImageIndexesPropertyEditor.GetAttributes
 0001:0001376C       ORCtrlsDsgn.TORImageIndexesPropertyEditor.GetProperties
 0001:000137A0       ORCtrlsDsgn.TORImageIndexesPropertyEditor.GetValue
 0001:00013754       ORCtrlsDsgn.TORImageIndexesPropertyEditor.Modified
 0001:000137B8       ORCtrlsDsgn.TORImageIndexesPropertyEditor.SetValue
 0001:0000181C       SysInit.@InitPkg
 0001:00001880       SysInit.@PackageLoad
 0001:0000188C       SysInit.@PackageUnload
 0001:0000170C       SysInit.AllocTlsBuffer
 0001:000017C8       SysInit.ExitProcessTLS
 0001:00001790       SysInit.ExitThreadTLS
 0001:000016D4       SysInit.FreeLibrary
 0001:00001718       SysInit.GetTlsSize
 0004:0000000C       SysInit.HInstance
 0001:000017EC       SysInit.InitializeModule
 0001:00001764       SysInit.InitProcessTLS
 0001:00001720       SysInit.InitThreadTLS
 0001:000016DC       SysInit.LocalAlloc
 0001:000016E4       SysInit.LocalFree
 0003:00000008       SysInit.Module
 0004:00000008       SysInit.ModuleIsLib
 0004:00000009       SysInit.ModuleIsPackage
 0003:00000004       SysInit.PtrToNil
 0001:000016EC       SysInit.TlsAlloc
 0004:00000010       SysInit.tlsBuffer
 0001:000016F4       SysInit.TlsFree
 0001:000016FC       SysInit.TlsGetValue
 0003:00000000       SysInit.TlsIndex
 0005:00000000       SysInit.TlsLast
 0003:00000020       SysInit.TlsProc
 0001:00001704       SysInit.TlsSetValue
 0001:000017F8       SysInit.UninitializeModule
 0004:00000000       Windows..3
 0001:00000364       Windows.CallNextHookEx
 0001:0000036C       Windows.DrawText
 0001:00000478       Windows.Finalization
 0001:0000032C       Windows.FreeLibrary
 0001:00000334       Windows.GetCurrentThreadId
 0001:00000374       Windows.GetCursorPos
 0001:0000037C       Windows.GetDC
 0001:00000384       Windows.GetDesktopWindow
 0001:0000038C       Windows.GetKeyState
 0001:00000394       Windows.GetScrollPos
 0001:0000039C       Windows.GetSystemMetrics
 0001:000003A4       Windows.GetTabbedTextExtent
 0001:00000344       Windows.GetTextExtentPoint32
 0001:0000034C       Windows.GetTextMetrics
 0001:0000033C       Windows.GetVersion
 0001:000003AC       Windows.GetWindowDC
 0001:000003B4       Windows.HideCaret
 0004:00000004       Windows.HtmlHelpModule
 0001:000003BC       Windows.InflateRect
 0001:000003C4       Windows.IntersectRect
 0001:000003CC       Windows.InvalidateRect
 0001:000003D4       Windows.KillTimer
 0001:0000043C       Windows.MakeLong
 0001:0000046C       Windows.MakeLParam
 0001:00000460       Windows.MakeWParam
 0001:000003DC       Windows.OffsetRect
 0001:00000448       Windows.PointToSmallPoint
 0001:000003E4       Windows.PostMessage
 0001:000003EC       Windows.PtInRect
 0001:000003F4       Windows.ReleaseDC
 0001:00000354       Windows.SelectObject
 0001:000003FC       Windows.SendMessage
 0001:0000035C       Windows.SetBkMode
 0001:00000404       Windows.SetTimer
 0001:0000040C       Windows.SetWindowPos
 0001:00000414       Windows.SetWindowsHookEx
 0001:0000041C       Windows.ShowWindow
 0001:00000424       Windows.SystemParametersInfo
 0001:0000042C       Windows.TabbedTextOut
 0001:00000434       Windows.UnhookWindowsHookEx
 0002:00000018       Windows.Windows


  Address             Publics by Value

 0001:0000032C       Windows.FreeLibrary
 0001:00000334       Windows.GetCurrentThreadId
 0001:0000033C       Windows.GetVersion
 0001:00000344       Windows.GetTextExtentPoint32
 0001:0000034C       Windows.GetTextMetrics
 0001:00000354       Windows.SelectObject
 0001:0000035C       Windows.SetBkMode
 0001:00000364       Windows.CallNextHookEx
 0001:0000036C       Windows.DrawText
 0001:00000374       Windows.GetCursorPos
 0001:0000037C       Windows.GetDC
 0001:00000384       Windows.GetDesktopWindow
 0001:0000038C       Windows.GetKeyState
 0001:00000394       Windows.GetScrollPos
 0001:0000039C       Windows.GetSystemMetrics
 0001:000003A4       Windows.GetTabbedTextExtent
 0001:000003AC       Windows.GetWindowDC
 0001:000003B4       Windows.HideCaret
 0001:000003BC       Windows.InflateRect
 0001:000003C4       Windows.IntersectRect
 0001:000003CC       Windows.InvalidateRect
 0001:000003D4       Windows.KillTimer
 0001:000003DC       Windows.OffsetRect
 0001:000003E4       Windows.PostMessage
 0001:000003EC       Windows.PtInRect
 0001:000003F4       Windows.ReleaseDC
 0001:000003FC       Windows.SendMessage
 0001:00000404       Windows.SetTimer
 0001:0000040C       Windows.SetWindowPos
 0001:00000414       Windows.SetWindowsHookEx
 0001:0000041C       Windows.ShowWindow
 0001:00000424       Windows.SystemParametersInfo
 0001:0000042C       Windows.TabbedTextOut
 0001:00000434       Windows.UnhookWindowsHookEx
 0001:0000043C       Windows.MakeLong
 0001:00000448       Windows.PointToSmallPoint
 0001:00000460       Windows.MakeWParam
 0001:0000046C       Windows.MakeLParam
 0001:00000478       Windows.Finalization
 0001:00000B4C       CommCtrl.TreeView_GetItem
 0001:00000B64       CommCtrl.TreeView_SetItem
 0001:000016D4       SysInit.FreeLibrary
 0001:000016DC       SysInit.LocalAlloc
 0001:000016E4       SysInit.LocalFree
 0001:000016EC       SysInit.TlsAlloc
 0001:000016F4       SysInit.TlsFree
 0001:000016FC       SysInit.TlsGetValue
 0001:00001704       SysInit.TlsSetValue
 0001:0000170C       SysInit.AllocTlsBuffer
 0001:00001718       SysInit.GetTlsSize
 0001:00001720       SysInit.InitThreadTLS
 0001:00001764       SysInit.InitProcessTLS
 0001:00001790       SysInit.ExitThreadTLS
 0001:000017C8       SysInit.ExitProcessTLS
 0001:000017EC       SysInit.InitializeModule
 0001:000017F8       SysInit.UninitializeModule
 0001:0000181C       SysInit.@InitPkg
 0001:00001880       SysInit.@PackageLoad
 0001:0000188C       SysInit.@PackageUnload
 0001:00001910       ORCtrls..TORStrings
 0001:00001D28       ORCtrls..TORListBox
 0001:000022C8       ORCtrls..TORDropPanel
 0001:00002474       ORCtrls..TORComboPanelEdit
 0001:000025DC       ORCtrls..TORComboEdit
 0001:0000283C       ORCtrls..TORComboBox
 0001:000032AC       ORCtrls..TORAutoPanel
 0001:00003414       ORCtrls..TOROffsetLabel
 0001:0000389C       ORCtrls..TORAlignButton
 0001:00003A8C       ORCtrls..TORAlignSpeedButton
 0001:00003BF0       ORCtrls..TORAlignEdit
 0001:00003E5C       ORCtrls..TCaptionTreeView
 0001:00004038       ORCtrls..TORTreeNode
 0001:0000412C       ORCtrls..TORTreeView
 0001:0000441C       ORCtrls..TORCBImageIndexes
 0001:000046AC       ORCtrls..TORCheckBox
 0001:00004A64       ORCtrls..TORListView
 0001:00004C34       ORCtrls..TORPopupMenu
 0001:00004D0C       ORCtrls..TORMenuItem
 0001:00004DE8       ORCtrls..TKeyClickPanel
 0001:00004F50       ORCtrls..TKeyClickRadioGroup
 0001:00005148       ORCtrls..TCaptionListBox
 0001:000053EC       ORCtrls..TCaptionCheckListBox
 0001:00005658       ORCtrls..TCaptionMemo
 0001:00005874       ORCtrls..TCaptionEdit
 0001:00005AA8       ORCtrls..TCaptionRichEdit
 0001:00005D04       ORCtrls..TCaptionComboBox
 0001:00005F58       ORCtrls..TCaptionListView
 0001:000061B8       ORCtrls..TCaptionStringGrid
 0001:000063A0       ORCtrls..TItemTip
 0001:000064F8       ORCtrls..TSizeRatio
 0001:00006574       ORCtrls.ClientWidthOfList
 0001:000065B8       ORCtrls.FontWidthPixel
 0001:000066BC       ORCtrls.FontHeightPixel
 0001:00006700       ORCtrls.HigherOf
 0001:0000670C       ORCtrls.LowerOf
 0001:00006718       ORCtrls.Piece
 0001:000067A8       ORCtrls.SetPiece
 0001:000068D0       ORCtrls.IntArrayToString
 0001:000069A0       ORCtrls.StringToIntArray
 0001:00006B0C       ORCtrls.StringBetween
 0001:00006B44       ORCtrls.ItemTipKeyHook
 0001:00006B78       ORCtrls.AddItemTipRef
 0001:00006BB0       ORCtrls.RemoveItemTipRef
 0001:00006BE0       ORCtrls.TItemTip.Create
 0001:00006C34       ORCtrls.TItemTip.Destroy
 0001:00006C70       ORCtrls.TItemTip.CreateParams
 0001:00006C9C       ORCtrls.TItemTip.Paint
 0001:00006D84       ORCtrls.TItemTip.Hide
 0001:00006DC8       ORCtrls.TItemTip.GetTabSettings
 0001:00006EF4       ORCtrls.TItemTip.UpdateText
 0001:0000719C       ORCtrls.TItemTip.Show
 0001:000074E8       ORCtrls.GetORCBBitmap
 0001:000075AC       ORCtrls.DestroyORCBBitmaps
 0001:000075E0       ORCtrls.TORStrings.Add
 0001:00007660       ORCtrls.TORStrings.Clear
 0001:00007690       ORCtrls.TORStrings.Create
 0001:000076E8       ORCtrls.TORStrings.Delete
 0001:00007720       ORCtrls.TORStrings.Destroy
 0001:00007754       ORCtrls.TORStrings.Get
 0001:0000777C       ORCtrls.TORStrings.GetCount
 0001:00007794       ORCtrls.TORStrings.GetObject
 0001:000077B4       ORCtrls.TORStrings.IndexOf
 0001:000077D4       ORCtrls.TORStrings.Insert
 0001:0000785C       ORCtrls.TORStrings.Put
 0001:000078DC       ORCtrls.TORStrings.PutObject
 0001:000078F8       ORCtrls.TORStrings.SetUpdateState
 0001:00007914       ORCtrls.TORStrings.Verify
 0001:00007D60       ORCtrls.TORListBox.Create
 0001:00007E60       ORCtrls.TORListBox.Destroy
 0001:00007EB4       ORCtrls.TORListBox.CreateParams
 0001:00007ECC       ORCtrls.TORListBox.CreateWnd
 0001:00007F24       ORCtrls.TORListBox.Loaded
 0001:00007F58       ORCtrls.TORListBox.DestroyWnd
 0001:00007F78       ORCtrls.TORListBox.TextToShow
 0001:00008074       ORCtrls.TORListBox.IsSynonym
 0001:00008168       ORCtrls.TORListBox.GetDisplayText
 0001:000081C4       ORCtrls.TORListBox.GetDynamicProperty
 0001:000081E8       ORCtrls.TORListBox.LBGetItemData
 0001:0000821C       ORCtrls.TORListBox.LBSetItemData
 0001:000082A8       ORCtrls.TORListBox.LBGetText
 0001:00008374       ORCtrls.TORListBox.LBGetTextLen
 0001:00008418       ORCtrls.TORListBox.LBAddString
 0001:00008504       ORCtrls.TORListBox.LBInsertString
 0001:00008610       ORCtrls.TORListBox.LBDeleteString
 0001:00008694       ORCtrls.TORListBox.LBResetContent
 0001:00008730       ORCtrls.TORListBox.LBSetCurSel
 0001:0000874C       ORCtrls.TORListBox.CMFontChanged
 0001:00008784       ORCtrls.TORListBox.WMKeyDown
 0001:000089A0       ORCtrls.TORListBox.WMLButtonDown
 0001:00008C54       ORCtrls.TORListBox.WMLButtonUp
 0001:00008C9C       ORCtrls.TORListBox.WMRButtonUp
 0001:00008D4C       ORCtrls.TORListBox.WMLButtonDblClk
 0001:00008F14       ORCtrls.TORListBox.WMCancelMode
 0001:00008F48       ORCtrls.TORListBox.WMMove
 0001:00008F68       ORCtrls.TORListBox.WMSize
 0001:00008FB0       ORCtrls.TORListBox.WMVScroll
 0001:00008FD4       ORCtrls.TORListBox.CMHintShow
 0001:00009034       ORCtrls.TORListBox.Click
 0001:00009050       ORCtrls.TORListBox.DoChange
 0001:000090BC       ORCtrls.TORListBox.DoEnter
 0001:000090FC       ORCtrls.TORListBox.DoExit
 0001:00009148       ORCtrls.TORListBox.DestroyItems
 0001:000091C0       ORCtrls.TORListBox.ToggleCheckBox
 0001:000092B4       ORCtrls.TORListBox.KeyPress
 0001:000092E8       ORCtrls.TORListBox.MouseDown
 0001:0000936C       ORCtrls.TORListBox.SetHintProperties
 0001:00009654       ORCtrls.TORListBox.MouseMove
 0001:00009870       ORCtrls.TORListBox.MeasureItem
 0001:00009914       ORCtrls.TORListBox.WMDestroy
 0001:00009940       ORCtrls.TORListBox.CNDrawItem
 0001:00009964       ORCtrls.TORListBox.DrawItem
 0001:00009DD0       ORCtrls.TORListBox.GetIndexFromY
 0001:00009E64       ORCtrls.TORListBox.SetFocusIndex
 0001:0000A13C       ORCtrls.TORListBox.UMShowTip
 0001:0000A274       ORCtrls.TORListBox.GetIEN
 0001:0000A324       ORCtrls.TORListBox.GetItemIEN
 0001:0000A3D4       ORCtrls.TORListBox.SelectByIEN
 0001:0000A438       ORCtrls.TORListBox.SetExactByIEN
 0001:0000A538       ORCtrls.TORListBox.GetItemID
 0001:0000A5D4       ORCtrls.TORListBox.SelectByID
 0001:0000A698       ORCtrls.TORListBox.GetReference
 0001:0000A734       ORCtrls.TORListBox.SetReference
 0001:0000A808       ORCtrls.TORListBox.AddReference
 0001:0000A878       ORCtrls.TORListBox.InsertReference
 0001:0000A8EC       ORCtrls.TORListBox.IndexOfReference
 0001:0000A99C       ORCtrls.TORListBox.GetTabPositions
 0001:0000A9D8       ORCtrls.TORListBox.SetTabPositions
 0001:0000AB84       ORCtrls.TORListBox.SetTabPosInPixels
 0001:0000AB9C       ORCtrls.TORListBox.SetTabStops
 0001:0000AD2C       ORCtrls.TORListBox.SupportsDynamicProperty
 0001:0000AD34       ORCtrls.TORListBox.SetHideSynonyms
 0001:0000ADF8       ORCtrls.TORListBox.SetSynonymChars
 0001:0000AE8C       ORCtrls.TORListBox.GetStyle
 0001:0000AE94       ORCtrls.TORListBox.SetStyle
 0001:0000AEC8       ORCtrls.TORListBox.SetDelimiter
 0001:0000AED8       ORCtrls.TORListBox.GetPieces
 0001:0000AEF8       ORCtrls.TORListBox.SetPieces
 0001:0000AF1C       ORCtrls.TORListBox.ResetItems
 0001:0000B134       ORCtrls.TORListBox.SetLongList
 0001:0000B16C       ORCtrls.TORListBox.AdjustScrollBar
 0001:0000B208       ORCtrls.TORListBox.CreateScrollBar
 0001:0000B2B8       ORCtrls.TORListBox.FreeScrollBar
 0001:0000B2DC       ORCtrls.TORListBox.ForDataUse
 0001:0000B594       ORCtrls.TORListBox.InitLongList
 0001:0000B728       ORCtrls.TORListBox.InsertSeparator
 0001:0000B7D0       ORCtrls.TORListBox.ClearTop
 0001:0000B834       ORCtrls.ClearLong
 0001:0000B924       ORCtrls.TORListBox.NeedData
 0001:0000BC40       ORCtrls.TORListBox.PositionThumb
 0001:0000BCF0       ORCtrls.TORListBox.ScrollTo
 0001:0000C1F8       ORCtrls.TORListBox.GetStringIndex
 0001:0000C340       ORCtrls.TORListBox.SelectString
 0001:0000C644       ORCtrls.TORListBox.SetCheckBoxes
 0001:0000C694       ORCtrls.TORListBox.SetFlatCheckBoxes
 0001:0000C6B0       ORCtrls.TORListBox.GetChecked
 0001:0000C6F8       ORCtrls.TORListBox.SetChecked
 0001:0000C78C       ORCtrls.TORListBox.GetCheckedState
 0001:0000C7C8       ORCtrls.TORListBox.SetCheckedState
 0001:0000C850       ORCtrls.TORListBox.GetMultiSelect
 0001:0000C858       ORCtrls.TORListBox.SetMultiSelect
 0001:0000C87C       ORCtrls.TORListBox.GetCheckedString
 0001:0000C924       ORCtrls.TORListBox.SetCheckedString
 0001:0000C9C0       ORCtrls.TORListBox.GetMItems
 0001:0000C9F8       ORCtrls.TORListBox.SetMItems
 0001:0000CA3C       ORCtrls.TORListBox.Clear
 0001:0000CA58       ORCtrls.TORListBox.SetBlackColorMode
 0001:0000CA60       ORCtrls.TORListBox.SetCaption
 0001:0000CB00       ORCtrls.TORListBox.GetCaption
 0001:0000CB1C       ORCtrls.DropDownPanelOpened
 0001:0000CB48       ORCtrls.DropDownPanelClosed
 0001:0000CB78       ORCtrls.TORDropPanel.BtnClicked
 0001:0000CBB0       ORCtrls.TORDropPanel.Create
 0001:0000CC28       ORCtrls.TORDropPanel.CreateParams
 0001:0000CC68       ORCtrls.TORDropPanel.GetButton
 0001:0000CD18       ORCtrls.TORDropPanel.ResetButtons
 0001:0000CD4C       ORCtrls.TORDropPanel.Resize
 0001:0000CDE4       ORCtrls.TORDropPanel.UpdateButtons
 0001:0000CF68       ORCtrls.TORDropPanel.WMActivateApp
 0001:0000D008       ORCtrls.TORComboEdit.CreateParams
 0001:0000D040       ORCtrls.TORComboEdit.WMKillFocus
 0001:0000D0BC       ORCtrls.TORComboEdit.WMSetFocus
 0001:0000D118       ORCtrls.TORComboBox.Create
 0001:0000D2BC       ORCtrls.TORComboBox.WMDestroy
 0001:0000D2EC       ORCtrls.TORComboBox.CMFontChanged
 0001:0000D304       ORCtrls.TORComboBox.WMMove
 0001:0000D320       ORCtrls.TORComboBox.WMSize
 0001:0000D338       ORCtrls.TORComboBox.WMTimer
 0001:0000D398       ORCtrls.TORComboBox.EditControl
 0001:0000D3AC       ORCtrls.TORComboBox.AdjustSizeOfSelf
 0001:0000D52C       ORCtrls.TORComboBox.DropButtonDown
 0001:0000D55C       ORCtrls.TORComboBox.DropButtonUp
 0001:0000D58C       ORCtrls.TORComboBox.DropDownStatusChanged
 0001:0000D66C       ORCtrls.TORComboBox.ClearDropDownStatus
 0001:0000D684       ORCtrls.TORComboBox.Destroy
 0001:0000D6B4       ORCtrls.TORComboBox.DoEnter
 0001:0000D6DC       ORCtrls.TORComboBox.UMGotFocus
 0001:0000D70C       ORCtrls.TORComboBox.DoExit
 0001:0000D754       ORCtrls.TORComboBox.LoadComboBoxImage
 0001:0000D7EC       ORCtrls.TORComboBox.Loaded
 0001:0000D808       ORCtrls.TORComboBox.FwdChange
 0001:0000D83C       ORCtrls.TORComboBox.FwdChangeDelayed
 0001:0000DB4C       ORCtrls.TORComboBox.FwdClick
 0001:0000DCA0       ORCtrls.TORComboBox.FwdDblClick
 0001:0000DCC4       ORCtrls.TORComboBox.FwdKeyDown
 0001:0000E0A0       ORCtrls.TORComboBox.FwdKeyPress
 0001:0000E110       ORCtrls.TORComboBox.FwdKeyUp
 0001:0000E17C       ORCtrls.TORComboBox.FwdMouseUp
 0001:0000E1A0       ORCtrls.TORComboBox.FwdNeedData
 0001:0000E218       ORCtrls.TORComboBox.SetDropDownCount
 0001:0000E224       ORCtrls.TORComboBox.SetDroppedDown
 0001:0000E488       ORCtrls.TORComboBox.SetEditRect
 0001:0000E558       ORCtrls.TORComboBox.SetEditText
 0001:0000E5FC       ORCtrls.TORComboBox.SetItemIndex
 0001:0000E6E0       ORCtrls.TORComboBox.SelectByIEN
 0001:0000E70C       ORCtrls.TORComboBox.SelectByID
 0001:0000E730       ORCtrls.TORComboBox.SetExactByIEN
 0001:0000E75C       ORCtrls.TORComboBox.SetStyle
 0001:0000E92C       ORCtrls.TORComboBox.StartKeyTimer
 0001:0000E99C       ORCtrls.TORComboBox.StopKeyTimer
 0001:0000E9C8       ORCtrls.TORComboBox.SupportsDynamicProperty
 0001:0000E9D0       ORCtrls.TORComboBox.AddReference
 0001:0000EA34       ORCtrls.TORComboBox.Clear
 0001:0000EA5C       ORCtrls.TORComboBox.ClearTop
 0001:0000EA6C       ORCtrls.TORComboBox.ForDataUse
 0001:0000EA7C       ORCtrls.TORComboBox.InitLongList
 0001:0000EACC       ORCtrls.TORComboBox.IndexOfReference
 0001:0000EB2C       ORCtrls.TORComboBox.InsertReference
 0001:0000EB94       ORCtrls.TORComboBox.InsertSeparator
 0001:0000EBA4       ORCtrls.TORComboBox.Invalidate
 0001:0000EC08       ORCtrls.TORComboBox.GetAutoSelect
 0001:0000EC18       ORCtrls.TORComboBox.GetColor
 0001:0000EC24       ORCtrls.TORComboBox.GetDelimiter
 0001:0000EC34       ORCtrls.TORComboBox.GetDisplayText
 0001:0000EC54       ORCtrls.TORComboBox.GetDynamicProperty
 0001:0000EC78       ORCtrls.TORComboBox.GetItemHeight
 0001:0000EC88       ORCtrls.TORComboBox.GetIEN
 0001:0000ECAC       ORCtrls.TORComboBox.GetItemID
 0001:0000ECC8       ORCtrls.TORComboBox.GetItemIEN
 0001:0000ECEC       ORCtrls.TORComboBox.GetItemIndex
 0001:0000ED00       ORCtrls.TORComboBox.GetItemTipEnable
 0001:0000ED10       ORCtrls.TORComboBox.GetItemTipColor
 0001:0000ED20       ORCtrls.TORComboBox.GetLongList
 0001:0000ED30       ORCtrls.TORComboBox.GetMaxLength
 0001:0000ED40       ORCtrls.TORComboBox.GetPieces
 0001:0000ED5C       ORCtrls.TORComboBox.GetReference
 0001:0000ED7C       ORCtrls.TORComboBox.GetSelLength
 0001:0000ED90       ORCtrls.TORComboBox.GetSelStart
 0001:0000EDA4       ORCtrls.TORComboBox.GetSelText
 0001:0000EDC4       ORCtrls.TORComboBox.GetShortCount
 0001:0000EDD4       ORCtrls.TORComboBox.GetSorted
 0001:0000EDE4       ORCtrls.TORComboBox.GetHideSynonyms
 0001:0000EDF4       ORCtrls.TORComboBox.GetSynonymChars
 0001:0000EE14       ORCtrls.TORComboBox.SetHideSynonyms
 0001:0000EE24       ORCtrls.TORComboBox.SetSynonymChars
 0001:0000EE74       ORCtrls.TORComboBox.GetTabPositions
 0001:0000EE90       ORCtrls.TORComboBox.GetTabPosInPixels
 0001:0000EEA0       ORCtrls.TORComboBox.GetText
 0001:0000EEBC       ORCtrls.TORComboBox.SelectAll
 0001:0000EECC       ORCtrls.TORComboBox.SetAutoSelect
 0001:0000EEDC       ORCtrls.TORComboBox.SetBlackColorMode
 0001:0000EF08       ORCtrls.TORComboBox.SetColor
 0001:0000EF40       ORCtrls.TORComboBox.SetDelimiter
 0001:0000EF50       ORCtrls.TORComboBox.SetItemHeight
 0001:0000EF60       ORCtrls.TORComboBox.SetItemTipEnable
 0001:0000EF70       ORCtrls.TORComboBox.SetItemTipColor
 0001:0000EF80       ORCtrls.TORComboBox.SetLongList
 0001:0000EF90       ORCtrls.TORComboBox.SetMaxLength
 0001:0000EFA0       ORCtrls.TORComboBox.SetPieces
 0001:0000EFB0       ORCtrls.TORComboBox.SetReference
 0001:0000F010       ORCtrls.TORComboBox.SetSelLength
 0001:0000F028       ORCtrls.TORComboBox.SetSelStart
 0001:0000F040       ORCtrls.TORComboBox.SetSelText
 0001:0000F050       ORCtrls.TORComboBox.SetSorted
 0001:0000F060       ORCtrls.TORComboBox.SetTabPositions
 0001:0000F070       ORCtrls.TORComboBox.SetTabPosInPixels
 0001:0000F080       ORCtrls.TORComboBox.SetText
 0001:0000F090       ORCtrls.TORComboBox.SetItems
 0001:0000F0A4       ORCtrls.TORComboBox.GetCheckBoxes
 0001:0000F0B4       ORCtrls.TORComboBox.GetChecked
 0001:0000F0C4       ORCtrls.TORComboBox.GetCheckEntireLine
 0001:0000F0D4       ORCtrls.TORComboBox.GetFlatCheckBoxes
 0001:0000F0E4       ORCtrls.TORComboBox.SetCheckBoxes
 0001:0000F2D8       ORCtrls.TORComboBox.SetChecked
 0001:0000F310       ORCtrls.TORComboBox.SetCheckEntireLine
 0001:0000F320       ORCtrls.TORComboBox.SetFlatCheckBoxes
 0001:0000F330       ORCtrls.TORComboBox.DropPanelBtnPressed
 0001:0000F398       ORCtrls.TORComboBox.GetCheckedString
 0001:0000F3B4       ORCtrls.TORComboBox.SetCheckedString
 0001:0000F3C4       ORCtrls.TORComboBox.SetCheckBoxEditColor
 0001:0000F3F8       ORCtrls.TORComboBox.SetListItemsOnly
 0001:0000F418       ORCtrls.TORComboBox.SetOnCheckedText
 0001:0000F480       ORCtrls.TORComboBox.SetTemplateField
 0001:0000F4C8       ORCtrls.TORComboBox.GetOnSynonymCheck
 0001:0000F4E0       ORCtrls.TORComboBox.SetOnSynonymCheck
 0001:0000F500       ORCtrls.TORComboBox.GetEnabled
 0001:0000F50C       ORCtrls.TORComboBox.SetEnabled
 0001:0000F548       ORCtrls.TORComboBox.GetEditBoxText
 0001:0000F658       ORCtrls.TORComboBox.UpdateCheckEditBoxText
 0001:0000F6D8       ORCtrls.TORComboBox.CheckBoxSelected
 0001:0000F70C       ORCtrls.TORComboBox.GetMItems
 0001:0000F714       ORCtrls.TORComboBox.SetCaption
 0001:0000F724       ORCtrls.TORComboBox.GetCaption
 0001:0000F740       ORCtrls.TORComboBox.GetCaseChanged
 0001:0000F750       ORCtrls.TORComboBox.SetCaseChanged
 0001:0000F760       ORCtrls.TORComboBox.GetLookupPiece
 0001:0000F770       ORCtrls.TORComboBox.SetLookupPiece
 0001:0000F780       ORCtrls.TSizeRatio.Create
 0001:0000F7F8       ORCtrls.TORAutoPanel.Destroy
 0001:0000F870       ORCtrls.TORAutoPanel.BuildSizes
 0001:0000F968       ORCtrls.TORAutoPanel.Loaded
 0001:0000F99C       ORCtrls.TORAutoPanel.DoResize
 0001:0000FB44       ORCtrls.TORAutoPanel.Resize
 0001:0000FB70       ORCtrls.TOROffsetLabel.Create
 0001:0000FBD0       ORCtrls.TOROffsetLabel.CMTextChanged
 0001:0000FBE8       ORCtrls.TOROffsetLabel.CMFontChanged
 0001:0000FC00       ORCtrls.TOROffsetLabel.AdjustSizeOfSelf
 0001:0000FCA0       ORCtrls.TOROffsetLabel.DoDrawText
 0001:0000FD40       ORCtrls.TOROffsetLabel.Paint
 0001:0000FDDC       ORCtrls.TOROffsetLabel.GetTransparent
 0001:0000FDE8       ORCtrls.TOROffsetLabel.SetTransparent
 0001:0000FE2C       ORCtrls.TOROffsetLabel.SetVertOffset
 0001:0000FE3C       ORCtrls.TOROffsetLabel.SetHorzOffset
 0001:0000FE4C       ORCtrls.TOROffsetLabel.SetWordWrap
 0001:0000FE64       ORCtrls.TORAlignButton.Create
 0001:0000FEB4       ORCtrls.TORAlignButton.CreateParams
 0001:0000FEFC       ORCtrls.TORAlignButton.SetAlignment
 0001:0000FF14       ORCtrls.TORAlignButton.SetLayout
 0001:0000FF2C       ORCtrls.TORAlignButton.SetWordWrap
 0001:0000FF44       ORCtrls.TORTreeNode.EnsureVisible
 0001:0000FFF4       ORCtrls.TORTreeNode.GetBold
 0001:00010030       ORCtrls.TORTreeNode.GetORTreeView
 0001:0001004C       ORCtrls.TORTreeNode.GetParent
 0001:00010068       ORCtrls.TORTreeNode.GetText
 0001:00010080       ORCtrls.TORTreeNode.SetBold
 0001:000100C4       ORCtrls.TORTreeNode.SetPiece
 0001:00010108       ORCtrls.TORTreeNode.SetStringData
 0001:000101B4       ORCtrls.TORTreeNode.SetText
 0001:000101C0       ORCtrls.TORTreeNode.UpdateText
 0001:00010250       ORCtrls.CalcShortName
 0001:0001047C       ORCtrls.TORTreeNode.SetCaption
 0001:0001052C       ORCtrls.TORTreeView.CNNotify
 0001:000105B8       ORCtrls.TORTreeView.Create
 0001:000105F8       ORCtrls.TORTreeView.CreateNode
 0001:00010634       ORCtrls.TORTreeView.FindPieceNode
 0001:00010694       ORCtrls.TORTreeView.FindPieceNode
 0001:0001077C       ORCtrls.TORTreeView.GetExpandedIDStr
 0001:00010878       ORCtrls.TORTreeView.SetExpandedIDStr
 0001:00010888       ORCtrls.TORTreeView.SetExpandedIDStr
 0001:00010A08       ORCtrls.TORTreeView.GetHorzScrollPos
 0001:00010A20       ORCtrls.TORTreeView.GetVertScrollPos
 0001:00010A38       ORCtrls.TORTreeView.RenameNodes
 0001:00010AF8       ORCtrls.TORTreeView.SetNodeDelim
 0001:00010B10       ORCtrls.TORTreeView.SetHorzScrollPos
 0001:00010B4C       ORCtrls.TORTreeView.SetNodePiece
 0001:00010B64       ORCtrls.TORTreeView.SetVertScrollPos
 0001:00010BA0       ORCtrls.TORTreeView.GetNodeID
 0001:00010BC8       ORCtrls.TORTreeView.GetNodeID
 0001:00010C8C       ORCtrls.TORTreeView.SetShortNodeCaptions
 0001:00010C9C       ORCtrls.TORCBImageIndexes.Create
 0001:00010D20       ORCtrls.TORCBImageIndexes.Destroy
 0001:00010D54       ORCtrls.TORCBImageIndexes.SetImages
 0001:00010D94       ORCtrls.RStr
 0001:00010DD0       ORCtrls.TORCBImageIndexes.IdxString
 0001:00010EB4       ORCtrls.TORCBImageIndexes.SetIdxString
 0001:00011014       ORCtrls.TORCBImageIndexes.ImageListChanged
 0001:00011048       ORCtrls.TORCBImageIndexes.Notification
 0001:00011078       ORCtrls.TORCBImageIndexes.SetCheckedDisabledIndex
 0001:0001108C       ORCtrls.TORCBImageIndexes.SetCheckedEnabledIndex
 0001:000110A0       ORCtrls.TORCBImageIndexes.SetGrayedDisabledIndex
 0001:000110B4       ORCtrls.TORCBImageIndexes.SetGrayedEnabledIndex
 0001:000110C8       ORCtrls.TORCBImageIndexes.SetUncheckedDisabledIndex
 0001:000110DC       ORCtrls.TORCBImageIndexes.SetUncheckedEnabledIndex
 0001:000110F0       ORCtrls.TORCheckBox.Create
 0001:0001114C       ORCtrls.TORCheckBox.ListViewCreate
 0001:00011198       ORCtrls.TORCheckBox.CreateCommon
 0001:000111C8       ORCtrls.TORCheckBox.Destroy
 0001:00011210       ORCtrls.TORCheckBox.GetImageIndexes
 0001:0001122C       ORCtrls.TORCheckBox.GetImageList
 0001:00011238       ORCtrls.TORCheckBox.SetImageIndexes
 0001:00011248       ORCtrls.TORCheckBox.SetImageList
 0001:00011258       ORCtrls.TORCheckBox.Toggle
 0001:000112E8       ORCtrls.TORCheckBox.CreateParams
 0001:00011304       ORCtrls.TORCheckBox.CMEnabledChanged
 0001:00011320       ORCtrls.TORCheckBox.CMFontChanged
 0001:0001133C       ORCtrls.TORCheckBox.CNDrawItem
 0001:00011358       ORCtrls.TORCheckBox.CNMeasureItem
 0001:0001137C       ORCtrls.TORCheckBox.GetDrawData
 0001:00011934       ORCtrls.TORCheckBox.DrawItem
 0001:00011D28       ORCtrls.TORCheckBox.SetGrayedStyle
 0001:00011D4C       ORCtrls.TORCheckBox.WMLButtonDblClk
 0001:00011D64       ORCtrls.TORCheckBox.WMSize
 0001:00011D8C       ORCtrls.TORCheckBox.BMSetCheck
 0001:00011E94       ORCtrls.TORCheckBox.SetWordWrap
 0001:00011EBC       ORCtrls.TORCheckBox.SetAutoSize
 0001:00011EE4       ORCtrls.TORCheckBox.SetBlackColorMode
 0001:00011F00       ORCtrls.TORCheckBox.AutoAdjustSize
 0001:000120D4       ORCtrls.TORCheckBox.GetCaption
 0001:000120EC       ORCtrls.TORCheckBox.SetCaption
 0001:00012158       ORCtrls.TORCheckBox.SetAllowAllUnchecked
 0001:00012168       ORCtrls.TORCheckBox.SetGroupIndex
 0001:00012198       ORCtrls.TORCheckBox.SyncAllowAllUnchecked
 0001:00012218       ORCtrls.TORCheckBox.SetParent
 0001:00012230       ORCtrls.TORCheckBox.SetRadioStyle
 0001:00012244       ORCtrls.TORCheckBox.SetAssociate
 0001:00012280       ORCtrls.EnableCtrl
 0001:0001231C       ORCtrls.TORCheckBox.UpdateAssociate
 0001:0001233C       ORCtrls.TORCheckBox.Notification
 0001:00012370       ORCtrls.TORCheckBox.SetFocusOnBox
 0001:00012384       ORCtrls.TORCheckBox.BMGetCheck
 0001:000123B0       ORCtrls.TORCheckBox.BMGetState
 0001:000123B4       ORCtrls.TORListView.WMNotify
 0001:0001247C       ORCtrls.TORListView.LVMSetColumn
 0001:00012530       ORCtrls.TORListView.LVMSetColumnWidth
 0001:000125E4       ORCtrls.TORComboPanelEdit.Destroy
 0001:0001261C       ORCtrls.TORComboPanelEdit.Paint
 0001:000126E4       ORCtrls.TKeyClickPanel.KeyDown
 0001:00012708       ORCtrls.TKeyClickRadioGroup.Click
 0001:00012740       ORCtrls.TKeyClickRadioGroup.Create
 0001:000127A0       ORCtrls.TKeyClickRadioGroup.KeyDown
 0001:00012810       ORCtrls.TCaptionListBox.DoEnter
 0001:00012834       ORCtrls.TCaptionListBox.GetCaption
 0001:00012860       ORCtrls.TCaptionListBox.GetDynamicProperty
 0001:00012884       ORCtrls.TCaptionListBox.MoveFocusUp
 0001:000128C0       ORCtrls.TCaptionListBox.MoveFocusDown
 0001:00012914       ORCtrls.TCaptionListBox.SetCaption
 0001:00012998       ORCtrls.TCaptionListBox.SupportsDynamicProperty
 0001:000129A0       ORCtrls.TCaptionListBox.WMKeyDown
 0001:00012A4C       ORCtrls.TCaptionListBox.WMMouseMove
 0001:00012B0C       ORCtrls.TCaptionListBox.WMRButtonUp
 0001:00012C40       ORCtrls.TCaptionCheckListBox.GetCaption
 0001:00012C6C       ORCtrls.TCaptionCheckListBox.GetDynamicProperty
 0001:00012C90       ORCtrls.TCaptionCheckListBox.SetCaption
 0001:00012D14       ORCtrls.TCaptionCheckListBox.SupportsDynamicProperty
 0001:00012D1C       ORCtrls.TCaptionMemo.GetCaption
 0001:00012D48       ORCtrls.TCaptionMemo.GetDynamicProperty
 0001:00012D6C       ORCtrls.TCaptionMemo.SetCaption
 0001:00012DF0       ORCtrls.TCaptionMemo.SupportsDynamicProperty
 0001:00012DF8       ORCtrls.TCaptionEdit.GetCaption
 0001:00012E24       ORCtrls.TCaptionEdit.GetDynamicProperty
 0001:00012E48       ORCtrls.TCaptionEdit.SetCaption
 0001:00012ECC       ORCtrls.TCaptionEdit.SupportsDynamicProperty
 0001:00012ED4       ORCtrls.TCaptionRichEdit.GetDynamicProperty
 0001:00012EFC       ORCtrls.TCaptionRichEdit.SupportsDynamicProperty
 0001:00012F04       ORCtrls.TCaptionTreeView.GetCaption
 0001:00012F1C       ORCtrls.TCaptionTreeView.GetDynamicProperty
 0001:00012F40       ORCtrls.TCaptionTreeView.SetCaption
 0001:00012FD0       ORCtrls.TCaptionTreeView.SupportsDynamicProperty
 0001:00012FD8       ORCtrls.TCaptionComboBox.GetCaption
 0001:00013004       ORCtrls.TCaptionComboBox.GetDynamicProperty
 0001:00013028       ORCtrls.TCaptionComboBox.SetCaption
 0001:000130AC       ORCtrls.TCaptionComboBox.SupportsDynamicProperty
 0001:000130B4       ORCtrls.TORAlignSpeedButton.Paint
 0001:0001312C       ORCtrls.GoodNotifyWinEvent
 0001:00013134       ORCtrls.TCaptionStringGrid.ColRowToIndex
 0001:00013184       ORCtrls.TCaptionStringGrid.GetDynamicProperty
 0001:000131AC       ORCtrls.TCaptionStringGrid.IndexToColRow
 0001:00013210       ORCtrls.TCaptionStringGrid.KeyUp
 0001:0001328C       ORCtrls.TCaptionStringGrid.SupportsDynamicProperty
 0001:00013294       ORCtrls.IsAMouseButtonDown
 0001:000132CC       ORCtrls.TORComboBox.SetNumForMatch
 0001:000132F4       ORCtrls.TORComboBox.SetUniqueAutoComplete
 0001:000132FC       ORCtrls.TORListBox.VerifyUnique
 0001:0001344C       ORCtrls.TORComboBox.SetTextAutoComplete
 0001:000134C8       ORCtrls.TCaptionListView.GetDynamicProperty
 0001:000134EC       ORCtrls.TCaptionListView.SupportsDynamicProperty
 0001:000134F4       ORCtrls.Finalization
 0001:00013564       ORCtrlsDsgn..TORImageIndexesPropertyEditor
 0001:00013654       ORCtrlsDsgn..TORImageIndexesElementPropertyEditor
 0001:00013754       ORCtrlsDsgn.TORImageIndexesPropertyEditor.Modified
 0001:00013760       ORCtrlsDsgn.TORImageIndexesPropertyEditor.GetAttributes
 0001:0001376C       ORCtrlsDsgn.TORImageIndexesPropertyEditor.GetProperties
 0001:000137A0       ORCtrlsDsgn.TORImageIndexesPropertyEditor.GetValue
 0001:000137B8       ORCtrlsDsgn.TORImageIndexesPropertyEditor.SetValue
 0001:000137C4       ORCtrlsDsgn.TORImageIndexesElementPropertyEditor.Create
 0001:00013810       ORCtrlsDsgn.TORImageIndexesElementPropertyEditor.ParentImgIdx
 0001:0001384C       ORCtrlsDsgn.TORImageIndexesElementPropertyEditor.GetAttributes
 0001:00013858       ORCtrlsDsgn.TORImageIndexesElementPropertyEditor.GetName
 0001:00013994       ORCtrlsDsgn.TORImageIndexesElementPropertyEditor.GetValue
 0001:00013A5C       ORCtrlsDsgn.TORImageIndexesElementPropertyEditor.SetValue
 0001:00013B10       ORCtrlsDsgn.Register
 0001:00013C18       ORCtrlsDsgn.Finalization
 0001:00013FC8       .ORCtrlLib2006.@GetPackageInfoTable
 0001:00013FD0       .ORCtrlLib2006.@PackageLoad
 0001:00013FDC       .ORCtrlLib2006.@PackageUnload
 0002:00000018       Windows.Windows
 0002:000001A4       ORCtrls.ORCtrls
 0002:00000204       ORCtrlsDsgn.ORCtrlsDsgn
 0002:0000020C       .ORCtrlLib2006..ORCtrlLib2006
 0003:00000000       SysInit.TlsIndex
 0003:00000004       SysInit.PtrToNil
 0003:00000008       SysInit.Module
 0003:00000020       SysInit.TlsProc
 0003:00000030       ORCtrls.ALPHA_DISTRIBUTION
 0003:000001C4       ORCtrls.CheckBoxImageResNames
 0003:00000204       ORCtrls.BlackCheckBoxImageResNames
 0003:00000244       ORCtrls.uDropPanelOpenCount
 0003:00000248       ORCtrls.ComboBoxImages
 0003:00000250       ORCtrls.BlackComboBoxImages
 0003:00000258       ORCtrls.ButtonAlignment
 0003:00000264       ORCtrls.ButtonWordWrap
 0003:0000026C       ORCtrls.ButtonLayout
 0004:00000000       Windows..3
 0004:00000004       Windows.HtmlHelpModule
 0004:00000008       SysInit.ModuleIsLib
 0004:00000009       SysInit.ModuleIsPackage
 0004:0000000C       SysInit.HInstance
 0004:00000010       SysInit.tlsBuffer
 0004:00000014       ORCtrls..03
 0004:00000018       ORCtrls.uKeyHookHandle
 0004:0000001C       ORCtrls.uItemTip
 0004:00000020       ORCtrls.uItemTipCount
 0004:00000024       ORCtrls.uNewStyle
 0004:00000028       ORCtrls.HintArray
 0004:0000002C       ORCtrls.ORCBImages
 0004:000000AC       ORCtrls.uOldShowHintsSetting
 0004:000000B0       ORCtrlsDsgn..3
 0005:00000000       SysInit.TlsLast


Bound resource files

ORCTRLS.RES
ORCtrlLib2006.res
ORCtrlsDsgn.dcr
ORCtrlLib2006.drf


Program entry point at 0002:0000020C
